:0A00000075817F7401F58F02002E58
:10002B000240A8C294D294C2A4D2A57532007533F3
:10003B000075340075350075360075370075630033
:10004B00756400754500754601754701756001754E
:10005B006101756201754800754900754A00754B61
:10006B0000754C01C233754D00755A0075590075FA
:10007B005C00755B007553007554007552F0754E3E
:10008B0000754F00755000755D00C20AC22EC20C80
:10009B00C210C211C214C215C212C213C20FC216B1
:1000AB00C217C218C219C21AC21BC21CC21DC21E61
:1000BB00C21FC220D209C234C235D236740090009E
:1000CB0030F0900031F0900032F0900033F090005F
:1000DB0034F07400900035F0900036F090027F748D
:1000EB0000F0A37404F0A37407F0A37409F090015B
:1000FB00207416F09001217401F012384012384C24
:10010B009001177401F09001227401F09001237497
:10011B0001F09001277401F09001187401F0900127
:10012B00247401F09001197401F090011A7401F01C
:10013B0090011B7401F090011F7401F090011C746D
:10014B0001F090011D7401F090011E7401F09001FB
:10015B00297401F0753C00753D0012094F7538008C
:10016B001204D912037A1204E67538001201FD123B
:10017B00408212074BC2A1120ABB120AC5120ACF48
:10018B00120AED120B7B120B991204BF1204D91237
:10019B0001FD1201FD753C30753D08123DEC753CBF
:1001AB0000753D00123D87124042121D8C121E47F6
:1001BB00122426C202C20312326C122063123808B8
:1001CB001231FC12349F1220C2900122E0B40306BC
:1001DB0012331B0201E650F81224C5121C64121FC5
:1001EB00C21224070201CB783279FF0000D9FCD868
:1001FB00F822786479FF0000D9FCD8F82278967938
:10020B0096D9FED8FA2278FF799BD9FED8FA2278B4
:10021B000A790AD9FED8FA22E627F5270809E63724
:10022B00F528782722C3E697F5270809E697F528DE
:10023B007827228627872908098628872A1202C34E
:10024B00782C22862C08862D08862E08862F872947
:10025B0009872A1202667827792E227530007531AC
:10026B00101202A812027912029CD531F422C3E5B6
:10027B002E9529E52F952AE5309400500122E52E85
:10028B009529F52EE52F952AF52FE5309400F530BD
:10029B0022B3E52733F527E52833F52822C3E52CD0
:1002AB0033F52CE52D33F52DE52E33F52EE52F33D8
:1002BB00F52FE53033F53022E5278529F0A4F52C11
:1002CB0085F02DE528852AF0A4F52E85F02FE5285D
:0A02DB008529F0A4252DF52DE52E50
:1002E50035F0F52EE52F3400F52FE527852AF0A406
:1002F500252DF52DE52E35F0F52EE52F3400F52FBE
:1003050022E538B4101120010ED201C28174C01249
:10031500034AD282C28222E538B4200FC28174809A
:1003250012034AD282C28275380022C201A200920B
:1003350081900000E5822538F582E012034AD282D9
:10034500C282053822F954F053800F4280D282C20E
:1003550082E9C454F053800F4280221201FD22121B
:1003650001FD1201FD1201FD1201FD1201FD120137
:10037500FD1201FD22C282120360120360C281C216
:10038500831201FDD282C287C286D285D284120130
:10039500FDC282120360C281C2831201FDD282C2F4
:1003A50087C286D285D2841201FDC282120360C241
:1003B50081C2831201FDD282C287C286D285D284D0
:1003C5001201FDC282120360C281C2831201FDD2F5
:1003D50082C287C286D285C2841201FDC2821203FF
:1003E50060C281C2831201FDD282C287C286D285D4
:1003F500C2841201FDC282120360C281C28312014E
:10040500FDD282D287C286C285C2841201FDC28214
:10041500120360C281C2831201FDD282C287C286E5
:10042500C285C2841201FDC282120360C281C283E9
:100435001201FDD282D287D286D285C2841201FDF5
:10044500C282120360C281C2831201FDD282C287B9
:10045500C286C285C2841201FDC282120360C281B6
:10046500C2831201FDD282C287C286C285D284129E
:1004750001FDC282120360C281C2831201FDD282D4
:10048500C287C286C285C2841201FDC28212036080
:10049500C281C2831201FDD282C287D286D285C2B1
:1004A500841201FDC282120360D2002205A2E493E8
:1004B500A305A2F0A3DBF505A222900F5005A2909B
:1004C50000007B200204B1900F7005A29000007B14
:1004D500200204B1900FC005A29000007B20020409
:1004E500B1C283C281744012034AD282C28212020F
:1004F50011D281740012034AD282C282120211D231
:1005050081741E12034AD282C282120211D28174F0
:100515001E12034AD282C282120211D281741E12A5
:10052500034AD282C282120211D281741E12034A78
:10053500D282C282120211D281741E12034AD28261
:10054500C282120211D281741E12034AD282C28261
:10055500120211C283C281744812034AD282C28236
:10056500120211D281740412034AD282C28212028B
:1005750011D281740E12034AD282C282120211D2A2
:1005850081741512034AD282C282120211D2817479
:100595000412034AD282C282120211D28174041259
:1005A500034AD282C282120211D281740412034A12
:1005B500D282C282120211D281740412034AD282FB
:1005C500C282120211D281740012034AD282C282FF
:1005D500120211C283C281745012034AD282C282AE
:1005E500120211D281740412034AD282C28212020B
:1005F50011D281740412034AD282C282120211D22C
:1006050081740412034AD282C282120211D2817409
:100615000412034AD282C282120211D281741512C7
:10062500034AD282C282120211D281740E12034A87
:10063500D282C282120211D281740412034AD2827A
:10064500C282120211D281740012034AD282C2827E
:0E065500120211C283C281745812034AD2826B
:10066300C282120211D281740412034AD282C2825C
:10067300120211D281740E12034AD282C282120272
:1006830011D281741512034AD282C282120211D28C
:1006930081740412034AD282C282120211D281747B
:1006A3001512034AD282C282120211D281740E122F
:1006B300034AD282C282120211D281740412034A03
:1006C300D282C282120211D281740012034AD282F0
:1006D300C282120211222430F02275F00A84AFF094
:1006E30075F00A84E5F02430F0EF2430A3F022758E
:1006F300F00A84AFF075F00A842430F0E5F024307A
:10070300A3F0EF2430A3F0221206F2A3742CF0EE30
:100713002430A3F022D281C2831201FDD282D28778
:10072300D286D285D2841201FDC282120360D281A5
:10073300C2831201FDD282D287D286D285D284129D
:1007430001FDC282120360221204D91201FD1201BB
:10075300FD1201FD1201FD1201FD1201FD1201FD49
:100763001204BF753C24753D001201FD1201FD7595
:100773003C30753D001201FD1201FD753C20753DB5
:10078300021201FD1201FD753C20753D081201FDA9
:100793001201FD753C20753D201201FD1201FD750E
:1007A3003C20753D801201FD1201FD753C20753D15
:1007B300101201FD1201FD753C20753D041201FD6F
:1007C3001201FD753CA0753D001201FD1201FD757E
:1007D3003C60753D001201FD1201FD753C28753D1D
:1007E300001201FD1201FD753C22753D001201FD51
:1007F3001201FD753C20753D001201FD1201FD75CE
:100803003C20753D001201FD1201FD753C20753D34
:10081300401201FD1201FD753C21753D001201FDE1
:100823001201FD753C20753D011201FD1201FD759C
:100833003C20753D001204CC1201FD1201FD120192
:10084300FD1201FD1201FD1201FD1201FD1201FD58
:100853001201FD1201FD1201FD1201FD1201FD1233
:1008630001FD1201FD1201FD1201FD1201FD120134
:10087300FD1201FD1204D91201FD1201FD1201FD49
:100883001201FD221201FD1201FD1201FD1201FDF3
:100893001201FD1201FD1201FD1201FD1201FD12F3
:1008A30001FD1201FD1201FD1201FD1201FD1201F4
:1008B300FD1201FD1201FD1201FD1201FD1201FDE8
:1008C3001201FD1201FD1201FD1201FD1201FD12C3
:1008D30001FD1201FD1201FD1201FD1201FD1201C4
:1008E300FD1201FD1201FD1201FD1201FD1201FDB8
:1008F3001201FD1201FD1201FD1201FD2220B204BD
:100903007539002220B103D2042275390122E53959
:10091300B53A0485393A22B4001920040A053B8507
:10092300393AD206D20222153BC20485393AD2069D
:10093300D2032220040A153B85393AD206D2032278
:10094300053BC20485393AD206D20222C2B3C2B4ED
:10095300C2B5E53CF4200E0244FE7F083392B6D2C2
:10096300B5C2B5DFF7B2B30000C2B3E53DF4200E64
:100973000244FE79083392B6C2B5D2B5D9F7D2B4E0
:100983000000C2B422C293D2937908C290A29133D9
:10099300D290D9F7F53EC293D2937908C290A2922E
:1009A30033D290D9F7F53F22E582C4540FF9E5839A
:1009B300C46922E5820303543FF9E583030354C06A
:1009C30069227A0CC2A6D2A3A2C133C933C9C2A376
:0E09D300DAF2F8D2A622C2A3C2A63392A7D2AD
:1009E100A3DAF5C2A31209C5E95403F9227A057401
:1009F100C01209D9F5838882227A0574C81209D9EF
:100A0100F5838882227A0574D01209D9F583888208
:100A1100227A0574D81209D9F58388822285823217
:100A210085833375340075350078327536787537BE
:100A310000793612023E8552367537037936120235
:100A41004EE6228582328583337534007535007810
:100A510032753604753700793612022386320886DC
:100A61003375340075350078327536E8753703799A
:100A71003612023E753655753721793612024EE629
:100A8100228582328583337534007535007832755D
:100A91003611753700793612024EE62222C2A0E8DD
:100AA100120AAFE9120AAFEA120AAFD2A0227B08FA
:100AB100D2A13392A2C2A1DBF7227840790F7A004A
:100AC100120A9E227869790F7A00120A9E2278779B
:100AD10079007A00120A9E22782F79FF7AF0120AA1
:100AE1009E22782F79807A00120A9E22782F79002F
:100AF1007A00120A9E22782FF97A00120A9E227831
:100B01002F791F7A80120A9E22782F793F7A00125C
:100B11000A9E22782F79FC7A00120A9E22E583C46C
:100B210054F0F9E582C4FA540F49F9EA54F0FA2273
:100B3100120B1E7800120A9E22120B1E7801120A55
:100B41009E22120B1E7802120A9E22120B1E78039D
:100B5100120A9E22120B1E78A0120B5E22C296E888
:100B6100120B6FE9120B6FEA120B6FD296227B0800
:100B7100D2A1339295C2A1DBF722782779007A00BE
:100B8100120B5E2278A079FF7AF0120B5E2278A018
:100B910079807A00120B5E2278A079007A00120B1C
:100BA1005E2278A0791F7A80120B5E2278A0793FAD
:100BB1007A00120B5E2278A079FC7A00120B5E2279
:100BC100F532753300783275362275370079361271
:100BD100023E868208868322F532753300783275AB
:100BE1003622753700793612023E868208868322C4
:100BF100120E82F532753300783275362A75370058
:100C0100793612023E868208868322F532753300D8
:100C11007832753620753700793612023E868208A1
:100C2100868322900030E004B410027400F090003A
:100C310020A98229F582E022900034E0FA90003167
:100C4100E004B40F0274FFF0900F30932A90003447
:100C5100F0900033E004B410027400F0F990003415
:100C6100E0FA900020E58229F582EAF02290003432
:100C7100E0FA900032E004B4110274FFF0900F3FEB
:100C8100932A900034F0120C5222120C2454016069
:100C910008120C24541F246022747F22F974FF89E6
:100CA100F084F5F0120C248422120C2475F02084B7
:100CB10022120C2475F03384240122120C2475F0C5
:100CC1002084240122120C2475F03F842401221275
:100CD1000C2475F03384240322120C2475F0108443
:100CE10022120C2475F01F8422120C2475F020842A
:100CF100F8120C2475F03F842822120C245401753B
:100D0100F00CA422120C2475F0558475F00CA42269
:100D1100B40101225003740122B4070122500122BF
:100D2100740722B40101225003740122B40A012282
:100D3100500122740A22B40101225003740122B429
:100D41000D0122500122740D22B4010122500374BD
:0E0D51000122B4100122500122741022B401BC
:100D5F0001225003740422B40401225001227401B1
:100D6F0022B40101225003740A22B40A0122500155
:100D7F0022740122B40101225003741822B4180105
:100D8F0022500122740122B4010122500374012266
:100D9F00B43A0122500122743A22B40101225003C5
:100DAF00740122B4460122500122744622B401017B
:100DBF00225003740122B404012250012274042230
:100DCF00B40101225003740122B405012250012203
:100DDF00740522B40101225003740122B4200122B0
:100DEF00500122742022B40101225003740122B455
:100DFF00020122500122740222B401012250037415
:100E0F000122B4020122500122740222B4010122F4
:100E1F005003740122B4050122500122740522B43B
:100E2F000001225003740022B405012250012274E4
:100E3F000522B40001225003740022B40301225092
:100E4F000122740322B4FF03740C22B40B0122504D
:100E5F000122740C22B4FF02EC22B43C0122500197
:100E6F0022EC22B4FF03740022B4030122500122AA
:100E7F00740322B46001224002746022B4FF037431
:100E8F000022B4240122500122742422B401012231
:100E9F005003740122B4180122500122741822B495
:100EAF000101225003740122B40201225001227465
:100EBF000222B40101225003740122B40201225014
:100ECF000122740222F990027AE0F55EE9B4010181
:100EDF00225003740122B55E0122500122E55E22E9
:100EEF00F990027AE0F55EE9B40101225003740132
:100EFF0022B55E0122500122740122B40101225059
:100F0F0003740422B4040122500122740122B4019B
:100F1F0001225003740122B40C0122500122740CDF
:100F2F0022037F2C0C0105712133E6FF0B57681844
:100F3F00BD09A60D004B5D263585B196114093C8AE
:100F4F00D3204620204C20204120204D202045201A
:100F5F002043484F5244204D414348494E4520328B
:100F6F0020202056455253494F4E20312E303320EA
:100F7F00202020286329323031362D32303137206E
:100F8F0020496E697420616C6C2044617461203F4C
:100F9F00204F4B20202020202020202020204E4F8B
:100FAF002020506C65617365207761697420212062
:100FBF002020202020202020202020202020202022
:100FCF002020202020202020202020202020202012
:100FDF00204D4F44452050524F4752414D4D2020F8
:100FEF00204D4F44453C3E202343302020524F4F4D
:100FFF005420205030312020234331202020202026
:10100F00202020503031204449523A646F776E20AF
:10101F004449563A6E6F2020234331200173636198
:10102F006C653A50303120202343312002736361C5
:10103F006C653A50303120202343312003736361B4
:10104F006C653A50303120202043484F52442020C5
:10105F004152502F514152504547494F2020515531
:10106F00414E54204C454E4748542053454C454320
:10107F00544C6973743A41303120202043484F5209
:10108F00444C6973743A4130312020204152502F23
:10109F0051202041322020553031203C20326E64C7
:1010AF003E3C63686F726420417270656767696F59
:1010BF003E3C7363616C6520417270656767696F51
:0E10CF003E3C737461626C2E5175616E7469E3
:1010DD007A653E3C636C6F636B205175616E74690C
:1010ED007A653E63686F72647363616C65207570B9
:1010FD0020646F776E616C7431616C743272616EE5
:10110D00646E6F202020646972656374207065724F
:10111D00204356202020207374657020627920733F
:10112D007465706F6666206F6E43484F5244202081
:10113D002020205343414C4520202020204B455951
:10114D004E4F54453A20204C4953543A41303120AA
:10115D0020534554555020202020204152504547C2
:10116D0047494F20205341564520202020202072F2
:10117D006F6F7420203173742020326E6420203301
:10118D007468205452414E53504F53453A202049D4
:10119D004E505554202020204F63746176652052A7
:1011AD00616E67654F6374617665205472616E730D
:1011BD00706F736520312D4F6374204469726563C0
:1011CD0074696F6E20322D4F6374204469726563AC
:1011DD0074696F6E20332D4F63742044697265639B
:1011ED0074696F6E20202053455454494E47534324
:1011FD00484F5244203E205530315343414C4520F9
:10120D003E205530312020204C495354203E204162
:10121D005072657373206B65792043484F5244219A
:10122D00202053544F52414745204F4B2021202021
:10123D002054554E452D4D4F444520204155544F7A
:10124D004C4F4144206C617374207361766564204A
:10125D004C6973742020202020202020204C69739D
:10126D00743A20415365742043562D4F5554733AAB
:10127D00202B38564B45594E4F54453A2020432389
:10128D00432044234420452046234620472347201E
:10129D004123412042030000000004000C000C0318
:1012AD00000C180C04000C182402000700070400A1
:1012BD00070E1502000500050400050A0F020004C3
:1012CD000004030004080C020003000303000306DE
:1012DD000C040003070E0400030A11040003060AA0
:1012ED000400030A0E040003070B030003060C049D
:1012FD000003070A0400030709030003070C03009A
:10130D0004070C0400040709040004070A04000480
:10131D00070B030005070C030002070C040004096A
:10132D000E030004080C030004060C040005070A54
:10133D00040004080A040004060A0400040B0E0449
:10134D0000040B0D0400040B0F040004070E040031
:10135D000B0E1104000B101504000B0E15040004E8
:10136D000B12030000000020202020202020202030
:10137D00554E49534F4E4F202020202020204F43C3
:10138D0054415645532031202020202020204F430A
:10139D0054415645532032202020202020204F43F9
:1013AD00544156455320332020202020202020203A
:1013BD00464946544820312020202020202020203E
:1013CD004649465448203220202020202020204607
:1013DD004F555254482031202020202020202046D7
:1013ED004F55525448203220202020205448495235
:1013FD0044206D616A20312020202020202041557D
:10140D00474D454E544544202020202054484952F4
:10141D0044206D696E203120202020202044494D2C
:10142D00494E495348454420202020204D494E4FD8
:10143D00522061646420392020202020204D494E07
:0E144D004F5220372F31312020202020204DFB
:10145B00494E4F522037206235202020202020205B
:10146B004D494E4F5220372F3920202020204D49F7
:10147B004E4F52206D616A203720202020202020E3
:10148B00204D494E4F522062352020202020202015
:10149B0020204D494E4F5220372020202020202045
:1014AB0020204D494E4F5220362020202020202036
:1014BB00202020204D494E4F52202020202020203C
:1014CB00202020204D414A4F522020202020202038
:1014DB0020204D414A4F5220362020202020202012
:1014EB0020204D414A4F52203720202020204D41B3
:1014FB004A4F52206D616A203720202020204D4119
:10150B004A4F5220737573203420202020204D41E8
:10151B004A4F522073757320322020202020202028
:10152B004D414A4F5220362F392020202020202099
:10153B00204D414A4F5220233520202020202020AF
:10154B00204D414A4F522062352020202020202060
:10155B004D414A4F5220372F342020202020204D40
:10156B00414A4F5220372023352020202020204D68
:10157B00414A4F5220372062352020202020202046
:10158B004D414A4F5220372F392020202020204D0B
:10159B00414A4F5220372062392020202020204DF5
:1015AB00414A4F52203720233920202020204D4103
:1015BB004A4F52206164642039202020204D414A3B
:1015CB004F5220372F392F31312020202020204D12
:1015DB00414A4F5220372F3133202020204D414A92
:1015EB004F5220372F392F313320202020204D41CF
:1015FB004A4F5220376220313120202020202020DA
:10160B002020554E49534F4E4F202020202020752F
:10161B007365722063686F72640800020305060726
:10162B00080B00000000060001040507080000007D
:10163B000000000500010307080000000000000087
:10164B000600030407090A0000000000000600035F
:10165B000506070A0000000000000700010405074B
:10166B00080B00000000000C000102030405060734
:10167B0008090A0B0500020407090000000000001E
:10168B0000070001040507080B000000000007001D
:10169B00010406080A0B0000000000050002050704
:1016AB000A00000000000000070002040507080AFA
:1016BB000000000000070003040607090A000000F1
:1016CB000000070002030607080B000000000005DE
:1016DB0000020307080000000000000005000105E0
:1016EB00060A0000000000000005000105070800C5
:1016FB0000000000000005000105070A00000000C3
:10170B0000000005000305070A00000000000000B0
:10171B0005000205070A000000000000000500029A
:10172B000407090000000000000007000204050682
:10173B00080A0000000000070001030406080A0065
:10174B0000000000070002040607080A0000000062
:10175B0000070002030507080B000000000007004C
:10176B0001030506090A000000000007000204053A
:10177B0008090B0000000000070002030607090A16
:10178B000000000000070001040507080A00000024
:10179B000000070003040607090B00000000000708
:1017AB000001030406080900000000000700020303
:1017BB000507090B000000000007000204050709DC
:0E17CB000B0000000000070002030507090ADA
:1017D9000000000000070001030507080A000000D7
:1017E9000000070002040607090B000000000007BB
:1017F9000002040507090A000000000007000203AF
:101809000507080A00000000000700010305060893
:101819000A0000000000070001030507090B00008A
:10182900000000070001030507080B000000000085
:101839000900020304060708090B0000000800015B
:1018490003040607090A0000000007000104050651
:10185900090A0000000000070002040607090A003F
:101869000000000005000103070800000000000057
:10187900000500020507090000000000000005003E
:101889000204070900000000000000050003050725
:101899000A0000000000000005000204060A00001A
:1018A9000000000000070001040507080A00000005
:1018B900000008000103040607090A0000000006E9
:1018C90000020406080A00000000000007000204E4
:1018D90006080A0B000000000020202020202020FC
:1018E90020416C67657269616E20202020202020CC
:1018F90020204172616269616E20202020202042EF
:10190900616C696E657369616E2020202020426CCC
:10191900756573206D616A6F722020202020426CEA
:10192900756573206D696E6F72202020202020203C
:1019390042797A616E74696E65202020202020200A
:101949004368726F6D617469632020202020202014
:1019590020446961746F6E696320446F75626C65B8
:10196900204861726D6F6E6963202020202020203D
:10197900456E69676D6174696320202020202020ED
:1019890020456779707469616E202020202020200D
:1019990048696E64757374616E2048756E6761720B
:1019A90069616E206D616A6F722048756E67617238
:1019B90069616E206D696E6F724A6170616E3A205D
:1019C90068697261796F7368694A6170616E3A69B1
:1019D9007761746F796F7368694A6170616E3A6B88
:1019E900756D6F69796F7368694A6170616E3A20C4
:1019F90020202020696E73656E4A6170616E3A20FD
:101A090020202020796F73656E4A6170616E3A20DB
:101A190020726974737573656E4A6170616E3A20DC
:101A290020202072796F73656E2020206D616A6FA6
:101A390072204C6F637269616E2020207375706526
:101A490072204C6F637269616E202020204C79648A
:101A590069616E206D696E6F724D696E6F72206873
:101A690061726D6F6E696320314D696E6F722068A6
:101A790061726D6F6E696320324D696E6F72206895
:101A890061726D6F6E696320334D696E6F72206884
:101A990061726D6F6E696320344D696E6F72206873
:101AA90061726D6F6E696320354D696E6F72206862
:101AB90061726D6F6E696320364D696E6F72206851
:101AC90061726D6F6E696320372020204D696E6FDA
:101AD90072206D656C6F6469634D6F64653A204966
:101AE9006F6E69616E2F4D616A4D6F64653A202092
:101AF900202020446F7269616E4D6F64653A202021
:101B090020506872796769616E4D6F64653A20206B
:101B19002020204C796469616E4D6F64653A204DCF
:101B290069786F6C796469616E4D6F64653A416576
:101B39006F6C69616E2F4D696E4D6F64653A202037
:0E1B490020204C6F637269616E4E6561706F93
:101B57006C6974616E206D616A6F724E6561706F3A
:101B67006C6974616E206D696E6F72202020202071
:101B770020204E696E6520546F6E6520202020203E
:101B870020204F637461746F6E69632020202020CA
:101B97002020204F7269656E74616C202020202000
:101BA7002020204F766572746F6E652020202020DC
:101BB70020202020202050656C6F672020202020C7
:101BC7002050656E7461746F6E69636D616A6F72C0
:101BD7002050656E7461746F6E69636D696E6F72A4
:101BE7002050656E7461746F6E6963202020202019
:101BF7002050726F6D6574686575732020202020F2
:101C0700202020205370616E6973682020202020D7
:101C170053796D6D6574726963616C202020202093
:101C2700202057686F6C65746F6E656C65616469B9
:101C37006E6757686F6C65746F6E65202020202073
:101C47002075736572207363616C65010000000085
:101C570001000000000000000000000000E53F3028
:101C6700E407121CA1121DD422121C77121C8C220D
:101C770020020122C205900117E004120D11F01293
:101C87001CE9C2022220030122C205900117E014B9
:101C9700120D11F0C203121CE922E53E30E10122C8
:101CA700E53E30E01530E31730E52DE53F30E7231B
:101CB70030E11130E21830E310227401021CE174A4
:101CC70002021CE17403021CE17404021CE17405A6
:101CD700021CE17406021CE17407900117F0121C44
:101CE700E922900117E01475F003A4901CF6730223
:101CF7001D0B021D1B021D2B021D3D021D56021D41
:101D070069021D767401900117F0121D8C12206371
:101D1700123808227402900117F0121D8C1224AB9E
:101D2700123824227403900117F0121D8CE54E120D
:101D370034C212352E227404900117F0121D8C1232
:101D47002960533C21533D41433C14433D282274B1
:101D570005900117F0121D8C533C21533D41433D23
:101D670028227406900117F0121D8C12283E227447
:101D770007900117F0121D8C533C21533D41433C02
:101D870002433D2822900117E0B401069011360264
:101D97001DC9B40206901140021DC9B40306901173
:101DA7004A021DC9B40406901154021DC9B40506A0
:101DB70090115E021DC9B40606901168021DC990F4
:101DC700117205A29000007B0A1204B1229001173C
:101DD700E01475F003A4901DE173021E0402221C97
:101DE7000233AA02288F023A1002280902385890B3
:101DF7000FC005A29000097B041204B122121E171E
:101E0700121E2F121E471221531236231235C322D8
:101E170020020122C205900120E004120D96F090E5
:101E27000120F0C202D2342220030122C205900110
:101E370020E014120D96F0900120F0C203D2342254
:101E4700900120121E54900120121FA822E0B42BEB
:101E570006901614021F9450F81475F006A4901EED
:101E67006973901374021F62901384021F629013A8
:101E770094021F629013A4021F629013B4021F62A0
:101E87009013C4021F629013D4021F629013E402DE
:101E97001F629013F4021F62901404021F629014D1
:101EA70014021F62901424021F62901434021F62EE
:101EB700901444021F62901454021F62901464022B
:0E1EC7001F62901474021F62901484021F6246
:101ED500901494021F629014A4021F629014B4021D
:101EE5001F629014C4021F629014D4021F629014E2
:101EF500E4021F629014F4021F62901504021F622F
:101F0500901514021F62901524021F629015340269
:101F15001F62901544021F62901554021F629015AE
:101F250064021F62901574021F62901584021F627D
:101F3500901594021F629015A4021F629015B402B9
:101F45001F629015C4021F629015D4021F6290157E
:101F5500E4021F629015F4021F6290160405A29018
:101F650000107B101204B11221A790000D7450F0DF
:101F75002205A29000107B101204B1900FC005A29B
:101F850090000A7B031204B190000D7450F02205F5
:101F9500A29000107B101204B11221A790000D74BD
:101FA50055F022E0B42B03021FB850FB90000E122F
:101FB50006DD22C3942A90000E1206DD222034018C
:101FC50022C234121FE41221E11220631238089054
:101FD5000120E0F56990015A123BB5E569F02290C0
:101FE5000120E0B42B0302202D50FB1475F005A44D
:101FF500FB9012A293FC0BEB93254EFD0BEB932567
:102005004EFE0BEB93254EFF0BEB93254E90003CBC
:10201500F090003BEFF090003AEEF0900039EDF0D3
:10202500900038ECF0F56022123D9E90027FE0FBB7
:10203500A3E0254EFCA3E0254EFDA3E0254EFEA31F
:10204500E0254E90003CF090003BEEF090003AED1C
:10205500F0900039ECF0900038EBF0F56022533C3D
:1020650021533D41E560B4000122B40108900039D7
:10207500E012210A22B4020F900039E012210A90E1
:10208500003AE012210A22B40316900039E0122129
:102095000A90003AE012210A90003BE012210A2240
:1020A500900039E012210A90003AE012210A9000CE
:1020B5003BE012210A90003CE012210A2290011710
:1020C500E0B40507300C04123B1F22900039E025CF
:1020D500532555120BF1120B3190003AE02553258B
:1020E50055120BF1120B3A90003BE0255325551282
:1020F5000BF1120B4390003CE025532555120BF1D3
:10210500120B4C2222F9E56375F00CA4C3C9991290
:102115000E5475F004A490211F73433C0222433CE6
:102125000422433C0822433C1022433C4022433CCA
:102135008022433D0222433D0422433D0822433D84
:102145001022433D2022433D8022433D0022900141
:1021550017E0B4010302215E22E53E30E10122E5EC
:102165003E30E20AE53F30E01FC210C211222010C6
:1021750016D210900142123BB5E004120D5DF090AD
:102185000124F01221D42222201116D211900142ED
:10219500123BB5E014120D5DF0900124F01221D42C
:1021A5002222900124E01475F006A49021B47390C6
:1021B500117C0221C99011810221C9901186022149
:1021C500C990118B05A29000087B051204B122125B
:1021D5001FE41221E112206312380822900124E045
:1021E500B4010122B40208900039E0240CF022B4B5
:1021F500030F900039E0240CF090003AE0240CF035
:1022050022900039E0240CF090003AE0240CF09084
:10221500003BE0240CF022122239122251122269CD
:10222500900FC005A29000087B051204B112362359
:102235001235C32220020122C205900121E00412B9
:0E2245000DA9F0900121F0C202D23522200333
:102253000122C205900121E014120DA9F090012181
:10226300F0C203D23522900121122279121DF69079
:1022730001211223ED22E0B43707901C42121F9470
:102283002250F7B42B0302228E400BC3942B75F01C
:1022930006A490239E731475F006A49022A2739053
:1022A30018E20223E99018F20223E99019020223AB
:1022B300E99019120223E99019220223E9901932B5
:1022C3000223E99019420223E99019520223E9906B
:1022D30019620223E99019720223E99019820223F9
:1022E300E99019920223E99019A20223E99019B205
:1022F3000223E99019C20223E99019D20223E9903B
:1023030019E20223E99019F20223E9901A02022347
:10231300E9901A120223E9901A220223E9901A3251
:102323000223E9901A420223E9901A520223E99008
:102333001A620223E9901A720223E9901A82022395
:10234300E9901A920223E9901AA20223E9901AB2A1
:102353000223E9901AC20223E9901AD20223E990D8
:102363001AE20223E9901AF20223E9901B020223E4
:10237300E9901B120223E9901B220223E9901B32EE
:102383000223E9901B420223E9901B520223E990A6
:102393001B620223E9901B720223E9901B82022332
:1023A300E9901B920223E9901BA20223E9901BB23E
:1023B3000223E9901BC20223E9901BD20223E99076
:1023C3001BE20223E9901BF20223E9901C02022381
:1023D300E9901C120223E9901C220223E9901C328B
:1023E3000223E9901C42121F7622E0B43703022332
:1023F300FD50FB90000E1206DD22C3943690000EB2
:102403001206DD2220350122C2351224261224AB06
:10241300123824900121E0F5699001A2123BB5E541
:1024230069F022900121E0B4370D123DB890003DD0
:10243300E0C3954EF5612250F112247D05A2900070
:102443003DF0F56112246C22B4370D123DD2900099
:102453004AE0C3954EF5622250F112247D05A29005
:10246300004AF0F56212246C22A305A20BEB93053C
:10247300A2254EF0A305A2DAF322B41303022485A6
:1024830050069016240224A2B42603022493500972
:1024930090171BC394130224A2901812C3942614FA
:1024A30075F00DA4FB93FA22533C21533D41900058
:1024B3003DE0FA700122A3E005A212210A05A2DA87
:1024C300F522120A121209B6B437030224DE500BA6
:1024D300D294533CFE533DFEC20922433C013009D2
:1024E3000122D2091546E5466001221227931225DF
:1024F3006E9001EA123BB5E0F546C294433D01E517
:1025030045B5470975450012330B02251250F512E4
:10251300253A12251B054522E02553254925561248
:10252300252622F9900117E0B40504300C0122E9B5
:10253300120BF1120B5522E54CB405041225572258
:10254300122547229000B7E5822545F582E58334BD
:1025530000F58322E547120C9DF5459000B7E5820F
:102563002545F582E5833400F58322900172123B01
:10257300B5E0B4010412258322B402031225AE226E
:10258300E54CB401079000B71225F422B40207907A
:1025930000B712262422B4030412268B22B40404A7
:1025A3001226A2229000B71225F422E54CB40107AB
:1025B3009000B71226D122B402079000B712270168
:0E25C30022B4030412276822B4040412277FF6
:1025D100229000B71226D122E56070057E017901B3
:1025E10022FEF922E560B402057E0279022240F959
:1025F100FEF9221225D9AB4B0B7A0005A2900039C6
:10260100122618EEF9EA240CFA900039DBF2E54BB8
:10261100048EF0A4F54722E02AA305A2F0A305A2A7
:10262100D9F5221225D9AB4BEB75F00CA4FA0B05A9
:10263100A2900038123BE6122653EEF9EAC3940C3D
:10264100FA900038123BE6DBEEE54B048EF0A4F580
:102651004722E02AFF123BD805A2EFF0A305A2D939
:10266100F1221225E519AB4BEB75F00CA4FA0B0521
:10267100A2900038123BE6122653EEF9EAC3940CFD
:10268100FA900038123BE6DBEE229000B71225F4F7
:1026910005A2122663E54775F002A4C39402F5472B
:1026A100229000B71225F405A2122624E54775F001
:1026B10002A4F54722E56170057E01790122FEF948
:1026C10022E561B402057E0279022240F9FEF92277
:1026D1001226B6AB4B0B7A0005A290003E1226F5EE
:1026E100EEF9EA240CFA90003EDBF2E54B048EF0A1
:1026F100A4F54722E02AA305A2F0A305A2D9F52259
:102701001226B6AB4BEB75F00CA4FA0B05A29000A8
:102711003D123BE6122730EEF9EAC3940CFA900021
:102721003D123BE6DBEEE54B048EF0A4F54722E0DB
:102731002AFF123BD805A2EFF0A305A2D9F122127C
:1027410026C219AB4BEB75F00CA4FA0B05A2900055
:102751003D123BE6122730EEF9EAC3940CFA9000E1
:102761003D123BE6DBEE229000B71226D105A21204
:102771002740E54775F002A4C39402F54722900073
:10278100B71226D105A2122701E54775F002A4F57B
:1027910047221227FC900127E0B401149001D212C4
:1027A1003BB5E0F54CE54A120E41F54B7549002267
:1027B100B402189001D2123BB5E0F54C754B00E51F
:1027C1004A120E2E75F00CA4F54922B4030EE54A07
:1027D100120DCFF54C754B0075490022B4040EE57E
:1027E1004A120DCFF54C754B0175490022E54A128D
:1027F1000DCFF54C754B0275490022120A06120ADB
:102801004475F00C84F54A22122810122827222040
:10281100020122900127E004120E1BF0900127F023
:1028210012283EC2022220030122900127E0141245
:102831000E1BF0900127F012283EC20322533C21C7
:10284100533D4190119A05A29000097B071204B1F2
:1028510012285522900127E0120E1BF01475F00684
:10286100A4902866739011A10228849011B10228C6
:10287100849011C10228849011D10228849011E121
:1028810002288405A29000107B101204B1221229A3
:102891002712289C122E4E1235C322E53E30E10448
:1028A1001228E8221228A922E53E30E222E53F3033
:1028B100E005C210C21122201014D210900129E0AB
:1028C10004120F1DF012403712296012326C2220BF
:1028D1001114D211900129E014120F1DF01240378A
:1028E10012296012326C22E53E30E222E53F30E0EF
:1028F10005C210C21122201014D21090011AE00456
:10290100120D83F0122B3D12296012326C2220111C
:1029110014D21190011AE014120D83F0122B3D1202
:10292100296012326C22E53E20E10122E53F30E6CA
:102931000AE53E30E417C214C2152220140ED21447
:0E294100900119E014120D70F012296022208E
:10294F00150ED215900119E004120D70F0122960C6
:10295F0022900119E0B40124122B54900FF405A218
:10296F009000107B011204B190012A122CA5900F38
:10297F00F505A29000147B011204B122B4022112BA
:10298F002B54900FF405A29000157B011204B11285
:10299F002CD6900FF505A290001A7B011204B122DC
:1029AF00B40328122B54900FF405A290001B7B0147
:1029BF001204B190015A123BB5E0122D06900FF59B
:1029CF0005A290001F7B011204B122B40404122B44
:1029DF008822B40904122B9F22B40A04122BDD2281
:1029EF00900172123BB5E0B40304122A9A2250FAF6
:1029FF00122A0322900119E0B40527122BF4900F2D
:102A0F00F405A29000107B011204B190018A122CE0
:102A1F00C5900FF505A29000147B011204B1122D81
:102A2F00D722B40621122BF4900FF405A290001BAD
:102A3F007B011204B1122DD7900FF505A290001F44
:102A4F007B011204B122B40721122C1E900FF40542
:102A5F00A29000137B011204B1122DF9900FF5050E
:102A6F00A29000187B011204B122122C1E900FF4B9
:102A7F0005A290001C7B011204B1900FF505A290E6
:102A8F00001F7B011204B1122E2F22900119E0B406
:102A9F000524122C45900FF405A29000107B011213
:102AAF0004B1900202122CC5900FF505A2900014EC
:102ABF007B011204B122B40627122C45900FF405A6
:102ACF00A290001B7B011204B1900232123BB5128F
:102ADF002D2C900FF505A290001F7B011204B1223F
:102AEF00B40724122C75900FF405A29000107B01EF
:102AFF001204B190021A122CC5900FF505A2900086
:102B0F00147B011204B122122C75900FF405A290C0
:102B1F00001B7B011204B190024A123BB5122D2CFF
:102B2F00900FF505A290001F7B011204B1229001B6
:102B3F001AE09000061206DD22900129E0142441CC
:102B4F00900005F022122B48122B3D90105605A233
:102B5F009000097B071204B1900FF605A2900010A8
:102B6F007B101204B190012A122CA5122CD69001C1
:102B7F005A123BB5E0122D0622122B48122B3D9014
:102B8F00105D05A29000097B071204B1122D52228D
:102B9F00122B48122B3D90107205A29000097B0753
:102BAF001204B1900FC005A29000107B0C1204B15B
:102BBF00900FF405A290001C7B011204B1122D821C
:102BCF00900FF505A290001F7B011204B122122B6A
:102BDF0048122B3D90107905A29000097B07120433
:102BEF00B1122D8D22122B48122B3D90106405A28D
:102BFF009000097B071204B190100605A2900010F7
:102C0F007B101204B190018A122CC5122DAE221224
:102C1F002B48122B3D90106405A29000097B0712E0
:102C2F0004B190101605A29000107B101204B1127F
:102C3F002DF9122E2F22122B48122B3D90106B05BF
:102C4F00A29000097B071204B190102605A29000F4
:102C5F00107B101204B1900202122CC59002321296
:102C6F003BB5122D2C22122B48122B3D90106B05C9
:102C7F00A29000097B071204B190103605A29000B4
:102C8F00107B101204B190021A122CC590024A1236
:102C9F003BB5122D2C22123BB5E075F00C84FEE5EE
:102CAF00F012358B05A29000117B021204B1EE9049
:0E2CBF0000131206D922123BB5E0900012124B
:102CCD0006DD900011742BF022900142123BB5E00D
:102CDD001475F006A4902CE67390117C022CFB90D9
:102CED001181022CFB901186022CFB90118B05A2F9
:102CFD009000167B041204B122E0B42B03022D1CAC
:102D0D0050FB90001D1206DD90001C7450F022C384
:102D1D00942A90001D1206DD90001C7455F022E0DF
:102D2D00B43703022D4250FB90001D1206DD9000BA
:102D3D001C7450F022C3943690001D1206DD9000D5
:102D4D001C7455F022900172123BB5E01475F0061B
:102D5D00A4902D62739010B0022D779010C0022DAB
:102D6D00779010D0022D779010E005A29000107B87
:102D7D00101204B12290027AE090001D1206DD229D
:102D8D0090027BE01475F006A4902D9A73901110AB
:102D9D00022DA390112005A29000107B101204B1FA
:102DAD0022900172123BB5E0B4010E9010F005A215
:102DBD009000167B051204B122B4020D9010F5059A
:102DCD00A29000167B051204B122900172123BB540
:102DDD00E0B4010A90015A123BB5122D0622B4023D
:102DED000A9001A2123BB5E0122D2C229001D212B5
:102DFD003BB5E01475F006A4902E09739010FA02FD
:102E0D002E249010FE022E24901102022E249011D9
:102E1D0006022E2490110A05A29000147B041204C0
:102E2D00B1229001EA123BB5E0B4010E90110E05EE
:102E3D00A290001D7B021204B12290001D1206DD2E
:102E4D0022900119E0B40107122EF8122F1422B4AA
:102E5D000207122F30122F4922B40307122F6212CC
:102E6D002F7B22B40407122F94122FAD22B4090721
:102E7D00122FC6122FD922B40A07122FEC122FFFD0
:102E8D0022900172123BB5E0B40304122ECC2250F5
:102E9D00FA122EA222900119E0B405071230121277
:102EAD00302E22B4060412304A22B407071230C65F
:102EBD001230DF22B408071230F81231102222909E
:102ECD000119E0B4050712312812314422B4060766
:102EDD0012316012317922B407071231921231AEDC
:102EED0022B408061231CA1231E3222002012290C7
:102EFD00012A123BB5E004120E8BF090012A122C20
:102F0D00A512326CC202222003012290012A123B2B
:102F1D00B5E014120E8BF090012A122CA512326C12
:102F2D00C2032220020122900142123BB5E004129D
:102F3D000D5DF0122CD612326CC20222200301223A
:102F4D00900142123BB5E014120D5DF0122CD61219
:102F5D00326CC203222002012290015A123BB5E0CD
:102F6D0004120D96F0122D0612326CC202222003AD
:102F7D00012290015A123BB5E014120D96F0122D5C
:102F8D000612326CC2032220020122900172123B02
:102F9D00B5E004120DBCF0122D5212326CC2022299
:102FAD0020030122900172123BB5E014120DBCF00A
:102FBD00122D5212326CC203222002012290027A8B
:102FCD00E004120E9BF0122D82C202222003012278
:102FDD0090027AE014120E9BF0122D82C203222071
:102FED0002012290027BE004120EAEF0122D8DC272
:102FFD0002222003012290027BE014120EAEF01289
:10300D002D8DC203222002012290018A123BB5E0D0
:10301D0004120E8BF090018A122CC512326CC20272
:10302D00222003012290018A123BB5E014120E8B6F
:0E303D00F090018A122CC512326CC203229050
:10304B000172123BB5E0B4010712306212307B22E1
:10305B001230941230AD222002012290015A123B01
:10306B00B5E004120D96F0122D0612326CC202223C
:10307B002003012290015A123BB5E014120D96F079
:10308B00122D0612326CC20322200201229001A2E1
:10309B00123BB5E004120DA9F0122D2C12326CC2AA
:1030AB000222200301229001A2123BB5E014120D63
:1030BB00A9F0122D2C12326CC20322200201229095
:1030CB0001D2123BB5E004120DCFF0122DF91232E2
:1030DB006CC20222200301229001D2123BB5E014F4
:1030EB00120DCFF0122DF912326CC2032220020105
:1030FB00229001EA123BB5E004120DE2F0F5461204
:10310B002E2FC20222200301229001EA123BB5E0CE
:10311B0014120DE2F0F546122E2FC20322200201EB
:10312B0022900202123BB5E004120E8BF0900202C9
:10313B00122CC512326CC202222003012290020211
:10314B00123BB5E014120E8BF0900202122CC5123A
:10315B00326CC2032220020122900232123BB5E0F4
:10316B0004120DA9F0122D2C12326CC20222200374
:10317B000122900232123BB5E014120DA9F0122D70
:10318B002C12326CC203222002012290021A123B33
:10319B00B5E004120E8BF090021A122CC512326C91
:1031AB00C202222003012290021A123BB5E0141234
:1031BB000E8BF090021A122CC512326CC203222015
:1031CB0002012290024A123BB5E004120DA9F01243
:1031DB002D2C12326CC202222003012290024A12C1
:1031EB003BB5E014120DA9F0122D2C12326CC20358
:1031FB002290027BE0B4010412320B2212324022E5
:10320B001209EE120A44B55D0122533DBFF55D1262
:10321B000ED490011AF012326C900117E0B4010435
:10322B0012206322B402041224AB22B40406122B24
:10323B003D122960221209EE1209B6B4370302328D
:10324B00545006533DBFC20D22433D40200D11D2B9
:10325B000D90011AE004120EEF90011AF0123221B8
:10326B0022D20A90012A123BB5E075F00C8485F04E
:10327B004E75F00CA4F55590015A123BB5E0900138
:10328B0020F0900142123BB5E0900124F0121FE4B4
:10329B001221E112380890018A123BB5E0F55690E5
:1032AB000202123BB5E0F55790021A123BB5E0F55E
:1032BB0058900172123BB5E0900122F012330BB41F
:1032CB0003041232EF2250FA1232D72220330302B8
:1032DB0032EE9001A2123BB5E0900121F0122426B0
:1032EB0012382422900232123BB5E0900121F012E9
:1032FB00242612382490024A123BB5E012244B22AA
:10330B00900122E0B40103C23322B40202D2332271
:10331B00900122E0B4030412334E22B4040312339F
:10332B002D22120A121209B6B4370302334150068A
:10333B00533CFEC20922433C0130090122D209123F
:10334B00334E22120A06120A44120E82B55A10206C
:10335B000A3722F55A85575990003D12337822507F
:10336B00F2F55A85585990004A1233782275F00CB1
:10337B008485F06975F00CA4FAE0F9A3E0C3954ECF
:10338B00B56903023394D9F322C20AF54D254E2AAF
:10339B0025592553122526C294433D01D23622E5E9
:1033AB003E20E101221233C312349FE54E1234C288
:0E33BB0012352EC202C20322E53E20E0057448
:1033C9000002342E20E205740102342E20E3057434
:1033D9000202342EE53F20E505740602342E20E072
:1033E90005740302342E20E105740402342E20E30F
:1033F90005740502342E20E205740702342E20E6F6
:1034090005740802342E20E705740902342EE53EBE
:1034190020E405740A02342E20E505740B02342ECB
:10342900E54EC22E22202E30D22E854E4FF54E1259
:10343900346212346E900125E54EF0A3F0F9900143
:103449002A123BB5E075F00C8475F00CA4254EF0FA
:1034590012256ED20A12326C22900038740412348A
:10346900791238082290003DE012348C1238242257
:10347900FA700122A3E0FC254EC3954F120E64F0A9
:10348900DAF222FA700122A3E0FC254EC3954F120D
:103499000E64F0DAF2221209FA120A44B43C030269
:1034A90034AE400122F553B5540122F55475F00CA0
:1034B90084F55C85F05BD20A22533C21533D4112CD
:1034C9000E5475F007A49034D373533D41433C0225
:1034D90022533D41433C0422533D41433C0822537E
:1034E9003D41433C1022533D41433C4022533D4121
:1034F900433C8022533C21433D0222533C21433D1E
:103509000422533C21433D0822533C21433D1022D0
:10351900533C21433D2022533C21433D8022533CCF
:1035290021533D4122900FC005A290000A7B04124D
:1035390004B1E54E12358B05A290000E7B021204F0
:10354900B190119005A29000107B0A1204B1900F5E
:10355900C005A290001A7B031204B1E55490001E25
:103569001206DD90001D742BF022E55B12358B05E8
:10357900A290001D7B021204B1E55C90001F1206A7
:10358900D92275F004A49035937390128A2290126F
:103599008C2290128E2290129022901292229012D6
:1035A9009422901296229012982290129A229012A6
:1035B9009C2290129E229012A022900117E0B40141
:1035C900030235DAB402030235DAB404030235DA48
:1035D90022E53E30E10122E53E30E40AE53F30E6EE
:1035E90016C212C2132220120DD212E56304120E62
:1035F90072F5631236112220130DD213E5631412EA
:103609000E72F56312361122900117E0B40104120B
:10361900206322B402031224AB22E53E20E10122F9
:1036290012364E12366212367612368A12369E12C9
:1036390036B21236C61236DA1236EE12370212379F
:103649001612372A22E53E30E003C20F22200F0866
:10365900D20F90005712373E22E53E30E203C216E0
:1036690022201608D21690005812373E22E53E3025
:10367900E303C21722201708D21790005912373EC8
:1036890022E53F30E003C21822201808D218900022
:103699005A12373E22E53F30E103C21922201908A8
:1036A900D21990005B12373E22E53F30E303C21A7C
:1036B90022201A08D21A90005C12373E22E53F30C8
:1036C900E503C21B22201B08D21B90005D12373E66
:1036D90022E53F30E203C21C22201C08D21C9000C4
:1036E9005E12373E22E53F30E603C21D22201D0847
:1036F900D21D90005F12373E22E53F30E703C21E1C
:1037090022201E08D21E90006012373E22E53E306C
:10371900E403C21F22201F08D21F90006112373E06
:1037290022E53E30E503C22022202008D220900065
:0E3739006212373E2205A2900117E0B401098A
:1037470005A2123B7212375F22B4020B05A2123B8D
:1037570096123B721237AE22E020E01DE560B404FA
:103767000F05A27B049000561237FD05A202377998
:1037770050EFE0D2E0F0023783C2E0F07C007B003C
:103787007A3090005705A290003905A2E030E00892
:103797000BEC05A2F0A305A2A30CDAF0900038EB1E
:1037A700F0F56012206322E020E01DE561B40C0F04
:1037B70005A27B0C9000861237FD05A20237C85080
:1037C700EFE0D2E0F00237D2C2E0F07C007B007A73
:1037D7003090008705A290003E05A2E030E0080B7C
:1037E700EC05A2F0A305A2A30CDAF090003DEBF0E4
:1037F700F5611224AB22A3E030E0FBDBF9C2E0F075
:1038070022123840900038E0FBA3E004FA05A290AA
:103817000056A3DAFD7401F005A2DBED2212384C45
:1038270090003DE0FBA3E004FA05A2900086A3DA2E
:10383700FD7401F005A2DBED22900057740079308A
:10384700F0A3D9FC2290008774007930F0A3D9FC4B
:103857002212386812393712398D1238A21239C933
:1038670022E53E20E10122E53F30E60AE53E30E46D
:1038770014C214C2152220140BD21490011CE01498
:10388700120F0AF02220150BD21590011CE004122A
:103897000F0AF02290000E1206DD2290011CE0B400
:1038A700010122B402071238C51238D822B403071F
:1038B7001238EB1238FE2212391112392422200253
:1038C700012290011DE004120D4AF012389BC2023A
:1038D700222003012290011DE014120D4AF0123834
:1038E7009BC203222002012290011EE004120D4A0E
:1038F700F012389BC202222003012290011EE0141D
:10390700120D4AF012389BC20322200201229001B5
:1039170029E004120F1DF0123981C202222003018F
:1039270022900129E014120F1DF0123981C20322DF
:1039370090011CE0B4010E9011F105A29000057BE7
:103947000B1204B122B4020E9011FC1239BE900181
:103957001DE012389B22B4030E9012071239BE9055
:10396700011EE012389B229012121239BE123981C1
:1039770090000E7420F012398122900129E014245E
:103987004190000FF022900035E060012290121D57
:1039970005A29000107B101204B12290122D05A2EF
:1039A7009000107B101204B122900FB005A2900076
:1039B700107B101204B12205A29000057B091204A6
:1039C700B122E53E30E003C20B22200B1BD20B12C3
:1039D70039B01201FDC2AF1239F0D2AF1203601233
:1039E70039A29000357404F02290011CE0B4010460
:1039F700123D3B22B40204123D6122B40304123D7E
:103A07007422124003123D3B22123A1A123A4D1207
:103A17003AA122E53E20E10122E53F30E60AE53EF4
:103A270030E414C214C2152220140BD21490011FC3
:103A3700E014120EC1F02220150BD21590011FE0E1
:103A470004120EC1F02290011FE0B4011190123D43
:103A570005A29000067B0A1204B1123AD6229012F0
:103A67004705A29000067B0A1204B1123A7622900B
:103A77000128E0B4010E90125105A29000107B10AE
:103A87001204B1221414244190001FF09012610512
:103A9700A29000107B0F1204B12290011FE0B40125
:103AA70007123AB6123AC622123B52123B62222042
:0E3AB700020122900118E004120D24F0C20258
:103AC5002220030122900118E014120D24F0C203F4
:103AD5002290127105A29000107B0D1204B1900185
:103AE50018E0B4011090113005A290001D7B03125F
:103AF50004B1C20C22141490001E1206D990127E35
:103B050005A290001D7B011204B190128005A290C0
:103B1500001F7B011204B1D20C22900118E014148D
:103B250075F00CA4F565120BF1120B31E565120B5E
:103B3500F1120B3AE565120BF1120B43E565120B19
:103B4500F1120B4CE565120BF1120B552220020107
:103B550022900128E004120D37F0C2022220030151
:103B650022900128E014120D37F0C20322E5637597
:103B7500F00CA48582328583337534007535007861
:103B850032F5367537007936120223868208868328
:103B95002285823285833375340075350078327518
:103BA50036307537007936120223868208868322DD
:103BB50085823285833375340075350078329001FE
:103BC5001AE014F536753700793612022386820815
:103BD500868322C3E5829401F582E5839400F5830B
:103BE50022E58229F582E5833400F5832285823238
:103BF500858333753400753500783290011DE014E6
:103C050075F005A4023C2385823285833375340023
:103C1500753500783290011EE01475F00DA4F53667
:103C250075370079361202238682088683228582BB
:103C350032858333753400753500783275F00502A9
:103C45003C5885823285833375340075350078326A
:103C550075F00DA4F5367537007936120223868284
:103C65000886832275325575330175340075350024
:103C7500783214F536753700793612023E86820899
:103C8500868322901C5205A29000007E1005A27F1B
:103C950005123CB8901C5205A2DEF22290003D05AB
:103CA500A29000A07E1005A2790D123CEF90003D78
:103CB500DEF62274009343D20205A2F0A375D25218
:103CC50075D2A2E5D220E0FB53D2FD05A2A3DFE326
:103CD5002290003D05A2901C577B0DE493A305A2FD
:103CE500F0A305A2DBF5123CA122E0A343D2020515
:103CF500A2F0A375D25275D2A2E5D220E0FB53D231
:103D0500FD05A2D9E52243D202438E20E0A353D27A
:103D1500FD538EDF05A2F0A305A2D9EA2243D20204
:103D2500438E20E0254EA353D2FD538EDF05A2F02E
:103D3500A305A2D9E822790A90012005A2900240A4
:103D450005A2123CEF22900125E54EF0A3E54FF0C8
:103D550022900125E0F54EA3E0F54F2290003805AD
:103D6500A2900000123BF205A27905123CEF2290C9
:103D7500003D05A29000A0123C0C05A2790D123C55
:103D8500EF22C2AF790A90024005A290012005A258
:103D9500123D0B123D56D2AF22C2AF900000C39424
:103DA5002B123C3305A290027F05A27905123D0B2B
:103DB500D2AF22C2AF9000A0C39437123C4705A2F0
:103DC50090003D05A2790D123D22D2AF22C2AF90DF
:103DD50000A0C39437123C4705A290004A05A2797A
:103DE5000D123D22D2AF22E53E30E10122753C1095
:103DF500900F9005A29000007B101204B1900FA0C7
:103E050005A29000107B101204B1E53E30E1FBE500
:103E15003F30E00630E632023E14E53F30E0FB126B
:103E250001FD1201FD900FB005A29000107B10124C
:0E3E350004B11201FD1201FDC2AF123C881251
:103E43003CD6123E5A123E9AD2AF22E53F30E6FBF1
:103E53001201FD1201FD229001207416F090012140
:103E63007401F09001227401F09001237401F09029
:103E730001247401F09001257400F0900126740070
:103E8300F09001277401F09001287401F09001294A
:103E93007401F0123D3B2290027A7418F090027B79
:103EA3007401F090012A7400123F2E90018A74006D
:103EB300123F2E9002027400123F2E90021A7400D9
:103EC300123F2E9001427401123F2E90015A741B2F
:103ED300123F2E9001727401123F2E9001A2742F93
:103EE300123F2E9001BA741B123F2E9001D274031D
:103EF300123F2E9001EA7401123F2E900232740198
:103F0300123F2E90024A7401123F2E123F12227466
:103F130001900129F0123C6912400E900129E0043E
:103F2300F0B40DF17401900129F0227B18F0A3DBAA
:103F3300FC22123FD574A0F9123FA2123FEBE566B3
:103F4300F9123FA2123FEBE567F9123FA2123FEBD2
:103F5300123FD574A1F9123FA2123FEB123F951203
:103F63003FF1123FC722E9FA123FD574A0F9123F7D
:103F7300A2123FF1E566F9123FA2123FF1E567F99C
:103F8300123FA2123FF1EAF9123FA2123FF1123F90
:103F9300C722D2A57808123FF7E933F9D8F8227877
:103FA30008E93392A5F9123FF7D8F6227B80DB02AA
:103FB300800E123FD574A0F9123FA2123FF140EEDA
:103FC300123FC722C2A500D2A4000000000000D205
:103FD300A522D2A500D2A4000000000000C2A500C3
:103FE3000000000000C2A422C2A5123FF722D2A5FE
:103FF300123FF7220000D2A4000000A2A5C2A4220F
:10400300900129E0123C6912400E2205A290012A78
:1040130005A27FD81240207F7D124020228583662F
:1040230085826705A2E0F9A305A2123F69123FAF9B
:10403300A3DFEA22900129E0123C6912405C22903E
:104043000128E0B40107900129E0024055149001D2
:1040530029F0123C6912405C2205A290012A05A2B4
:104063007FD812406E7F7D12406E228583668582E3
:1040730067123F35A3E905A2F0A305A2DFED227580
:10408300402875410475427D75430275440A90FFCB
:104093009C8582CA8583CB8582CC8583CD43C80426
:1040A300D2ADD2AF22C0E0C0D0E582C0E0E583C08C
:1040B300E0D2D4C2D3C2CFD54046754028120306FE
:1040C300120900120911B20E12094F30360DD544F0
:1040D3000A754405D294533DFEC236D5412275413B
:1040E30006120988120C39120C6ED542137542322E
:1040F300900035E0600214F0D54305754314B20512
:0D410300D0E0F583D0E0F582D0D0D0E032DE
:00000001FF
